:0600000000F014EF00F017
:0400080082EF02F091
:10001800D8CFFDF0E0CF10F0FACFFCF048EF06F0B3
:1000280000EE85F0240EEE6AE806FDE1106A0F6A1C
:1000380000EEAAF0370EEE6AE806FDE100EEA9F040
:10004800C60EF66E040EF76E0900F5CFEEFF87EFC9
:0200580002F0B4
:10010000506963504F562076320000000000000016
:10011000005F00000007000700147F147F14242AEA
:100120007F2A12C4C81026463649552250000503BE
:100130000000001C2241000041221C0014083E085F
:100140001408083E0808000050300010101010106D
:10015000006060000020100804023E5149453E0046
:10016000427F400042615149462141454B311814BC
:10017000127F1027454545393C4A494930017109EC
:1001800005033649494936064949291E00363600D5
:1001900000005636000008142241001414141414F0
:1001A00000412214080201510906324959513E7E8C
:1001B0001111117E7F494949363E414141227F411B
:1001C00041221C7F494949417F090909013E4149B2
:1001D000497A7F0808087F00417F41002040413F65
:1001E000017F081422417F404040407F020C027F83
:1001F0007F0408107F3E4141413E7F090909063EC8
:100200004151215E7F091929464649494931010179
:100210007F01013F4040403F1F2040201F3F4038AA
:10022000403F63140814630708700807615149458B
:1002300043007F414100552A552A550041417F0026
:10024000040201020440404040400001020400203A
:10025000545454787F484444383844444420384403
:1002600044487F3854545418087E0901020C5252F5
:10027000523E7F0804047800447D40002040443D05
:10028000007F1028440000417F40007C041804785F
:100290007C0804047838444444387C141414080856
:1002A0001414187C7C080404084854545420043F57
:1002B0004440203C4040207C1C2040201C3C4030DE
:1002C000403C44281028440C5050503C4464544C4A
:1002D000440D0A546578743A20000D0A0D0A4D65E4
:1002E00073673A20000D0A506963504F56207632EA
:1002F0000D0A5075736820454E5445520D0A000092
:100300000000000000005F00000007000700147FED
:10031000147F14242A7F2A12C4C810264636495551
:1003200022500005030000001C2241000041221C55
:100330000014083E081408083E0808000050300069
:100340001010101010006060000020100804023E21
:100350005149453E00427F4000426151494621419A
:10036000454B311814127F1027454545393C4A4901
:100370004930017109050336494949360649492979
:100380001E003636000000563600000814224100D8
:1003900014141414140041221408020151090632E5
:1003A0004959513E7E1111117E7F494949363E41DE
:1003B0004141227F4141221C7F494949417F09092E
:1003C00009013E4149497A7F0808087F00417F4181
:1003D000002040413F017F081422417F40404040BF
:1003E0007F020C027F7F0408107F3E4141413E7F27
:1003F000090909063E4151215E7F091929464649EE
:1004000049493101017F01013F4040403F1F2040E9
:10041000201F3F4038403F631408146307087008EA
:10042000076151494543007F414100552A552A55EE
:100430000041417F0004020102044040404040006E
:100440000102040020545454787F4844443838440E
:10045000444420384444487F3854545418087E0992
:1004600001020C5252523E7F0804047800447D4041
:10047000002040443D007F1028440000417F4000A0
:100480007C041804787C0804047838444444387C9C
:1004900014141408081414187C7C08040408485424
:1004A000545420043F4440203C4040207C1C2040C9
:1004B000201C3C4030403C44281028440C505050F4
:1004C0003C4464544C440100F2A417D0380ED66E5C
:1004D000D76A872B000E8823852B8623892B8A23B6
:1004E000010E865DF40ED8B4855D06E380A8A96B85
:1004F00000EE85F0EE6AEE6AF294FEC0EAFFFFC0FD
:10050000E9FF1100E9CFFFF0EACFFEF0DDD73DD8DB
:10051000800E8B6F250E8C6F8D6B8E6B8DEC04F0C7
:10052000AB0E9E6F000E9F6FAAC0E8FF4FEC05F068
:10053000AB0E8B6F000E8C6F47EC04F0A95323E1D8
:10054000AA2B070EAA6501D0AA6BAB0E9E6F000EF8
:100550009F6FAAC0E8FF4FEC05F0AAC001F0010EA2
:10056000006E012A02D0D8900036012EFCD7005030
:10057000ACEC03F09E0E9E6F1B0E9F6FDBEC06F043
:10058000010EE8CFA9F015D8D3D7F29EF20ED36EA4
:100590007F0EC16EF80E926E130E936ED59E380EBE
:1005A000D66ED76AF294CF0ED56EF28AF28CF28EA6
:1005B00012008C6B010E8B6FC30E8A5D510ED8B486
:1005C000895D0AE3E50E9E6F020E9F6FF9EC04F061
:1005D00000EE89F0EE6AEE6A83EC04F00009D8B40C
:1005E00012000AD0CFEC04F08D6F8D510D0A03E09C
:1005F0008D510A0AD8B48B6B83EC04F00009F2E148
:100600008B51D8A41200AAC001F0010E006E012A7D
:1006100002D0D8900036012EFCD70050ACEC03F08D
:10062000DC0E9E6F020E9F6FF9EC04F0AB0E9E6F16
:10063000000E9F6FF9EC04F0D10E9E6F020E9F6FBB
:10064000F9EC04F08B6B8D0E9E6F000E9F6FE2EC49
:1006500004F0006E00C002F0036A0350021039E19A
:10066000A953F1E1AA2B070EAA6501D0AA6BAB0E24
:100670009E6F000E9F6FAAC0E8FF4FEC05F0AAC066
:1006800001F0010E006E012A02D0D8900036012E32
:10069000FCD70050ACEC03F0DA0E9E6F020E9F6F99
:1006A000F9EC04F0AB0E9E6F000E9F6FF9EC04F0B6
:1006B0009E0E9E6F1B0E9F6FDBEC06F08C6BD10EB7
:1006C0009E6F020E9F6FF9EC04F0010EE8CFA9F0C7
:1006D000BAD78D510D0A03E08D510A0A0AE1010EC5
:1006E0008B6F8C5100EE8EF0E926000EEA22EF6E41
:1006F00016D01F0E8D6510D07B0E8D610DD08D51E3
:10070000B8EC04F08C5100EE8EF0E926000EEA22DF
:100710008DC0EFFF8C2B03D0070EB8EC04F08B518B
:1007200092E0FC0E9E6F020E9F6FF9EC04F08C516C
:10073000D8B412008E0E9E6F000E9F6FAAC0E8FF05
:10074000A4EC05F0AB0EA26F000EA36F8E0EA46F8B
:10075000000EA56FECEF06F0D96ED9CF00F0003097
:1007600002E3808001D08090D9CF00F0020E001605
:10077000010E016ED8900032012EFCD7003002E34A
:10078000808201D08092D9CF00F0040E0016020EB4
:10079000016ED8900032012EFCD7003002E3818632
:1007A00001D08196D9CF00F0080E0016030E016E1D
:1007B000D8900032012EFCD7003002E3818401D0B2
:1007C0008194D9CF00F0100E0016003A0F0E0016DB
:1007D000003002E3818E01D0819ED9CF00F0200E3F
:1007E0000016050E016ED8900032012EFCD70030A5
:1007F00002E3818C01D0819CD9CF00F0400E00161D
:10080000060E016ED8900032012EFCD7003002E3B4
:10081000818A01D0819AD9CF00F0800E0016070E90
:10082000016ED8900032012EFCD7003002E38084A4
:1008300001D08094190E9E6F9F6BDBEF06F0D96E8E
:10084000D9508F6F200ED96001D003D07A0ED964B1
:1008500002D0550E81D7906B8F51050D9051F32624
:10086000000EF422F350FF0FF66EF450F76E020EF6
:10087000F722600EF626FF0EF7220800F5506CDF17
:10088000902B040E9065E8D7000E66D78B008D6B19
:100890008E6B8BC000F08CC001F08D5100268E5104
:1008A000012200C0F6FF01C0F7FF000EF76403D07D
:1008B0000800F55005D0F6CFE9FFF7CFEAFFEF507B
:1008C00000091BE08BC000F08CC001F08D510026A8
:1008D0008E51012200C0F6FF01C0F7FF000EF76441
:1008E00003D00800F55005D0F6CFE9FFF7CFEAFFB7
:1008F000EF50A5DF8D4B8E2BCCD7F40E9E6F010EE3
:100900009F6FDBEF06F0BCC0E8FF12009D9ABC6B46
:10091000BB6BBD6B9D8A12008B00AC98AC84040E3F
:100920008BC000F08CC001F08DC002F08EC003F0CF
:1009300040EC07F000C004F001C005F002C006F072
:1009400003C007F0006A120E016E7A0E026E000EEE
:10095000036A7FEC06F00050AF6EAC8AAB88AB8EBA
:10096000939293889F989D989F9A9D8AD08E12000B
:10097000D96EBFC0E8FF100AFCE09D98C0C0E8FF38
:1009800000EED1F0E926000EEA22D9CFEFFFC02910
:100990000F0BE8CFC0F0010EBF2B9D881200BC5397
:1009A000FEE0BBC0E8FF00EEC1F0E926000EEA223F
:1009B000EF50D96EBB290F0BE8CFBBF0BC07D95065
:1009C00012009E00BC5301E1000CBBC0E8FF10EE1A
:1009D000C1F0E126000EE2229EC0E9FF9FC0EAFFBF
:1009E000E7CFEFFFBB290F0BE8CFBBF0BC07010C33
:1009F0009E009F519E11D8B412009EC0F6FF9FC06A
:100A0000F7FF000EF76403D00800F55005D0F6CFCD
:100A1000E9FFF7CFEAFFEF500009D8B412009EC0FB
:100A2000F6FF9FC0F7FF9E4B9F2B000EF76403D08D
:100A30000800F55005D0F6CFE9FFF7CFEAFFEF50F9
:100A400097DFD7D7A700BF5301E1000CBEC0E8FF76
:100A500010EED1F0E126000EE222A7C0E9FFA8C007
:100A6000EAFFE7CFEFFFBE290F0BE8CFBEF0BF07CD
:100A7000010CD96EBCC0E8FF100A01E1000CBDC03A
:100A8000E8FF00EEC1F0E926000EEA22D9CFEFFF21
:100A9000BD290F0BE8CFBDF0BC2B010C9E00A06F51
:100AA000070EA06501D0A06BA039F00BA16FA0517B
:100AB000100D0F0EF326000EF422A1C000F0016A03
:100AC0000150800A026EF450800A025C02E1F35089
:100AD000005C30E2A151A36FA46B4CEC07F0006EF8
:100AE000A1510F0B9E25E96E000E9F21EA6E00C0FA
:100AF000EFFFA1510F0B9E25E96E000E9F21EA6EBC
:100B0000EF50D8B41200A1510F0B9E25E96E000ED4
:100B10009F21EA6EEF50006E00280AE19EC0A2F00D
:100B20009FC0A3F0000EA46F010EA56FECEF06F0BE
:100B3000A12BBDD700EE0FF09E51E9269F51EA226E
:100B4000000EEF6A12009E00D96ED938F00BA26F2A
:100B5000A2510F0FA06FA16BA251A36FA46BA15163
:100B60009E25E96E000E9F21EA6EEF50A56F19ECED
:100B700007F0A251A36FA46B4CEC07F0016EA151DA
:100B80009E25E96E000E9F21EA6EEF50006E00C0B8
:100B900002F0036A01C0E8FF021801E10352DCE140
:100BA000A1519E25E96E000E9F21EA6EEF5005E0EF
:100BB000A12BA22BA051A25DCFE3A251A36FA46BE6
:100BC000A56B19EC07F0A251A36FA46B4CEC07F0D6
:100BD000006E00C002F0036A03500210D8B4120085
:100BE000ECD79EB89DA811D0A60EA76F000EA86FD7
:100BF00023EC05F0006E00C002F0036A03500210FF
:100C000003E0A6C0ADFF01D09D989EBA9DAA03D077
:100C1000AE5039EC05F0E1C0F3FFE2C0F4FFE3C0F1
:100C2000F5FFE4C0F6FFE5C0F7FFE6C000F0E7C05F
:100C300001F0E8C002F0E9C003F0EAC004F0EBC044
:100C400005F0ECC006F0EDC007F0EEC008F0EFC014
:100C500009F0F0C00AF0F1C00BF0F2C00CF0F3C0E4
:100C60000DF0F4C00EF0F5C0DAFFF6C0D9FFF7C002
:100C7000E2FFF8C0E1FFF9C0EAFFFAC0E9FFFBC0FC
:100C8000E8FFFCC0FAFF10C0E0FFFDC0D8FF100075
:100C9000E8CFFBF0E9CFFAF0EACFF9F0E1CFF8F0D6
:100CA000E2CFF7F0D9CFF6F0DACFF5F00EC0F4F0DE
:100CB0000DC0F3F00CC0F2F00BC0F1F00AC0F0F080
:100CC00009C0EFF008C0EEF007C0EDF006C0ECF090
:100CD00005C0EBF004C0EAF003C0E9F002C0E8F0A0
:100CE00001C0E7F000C0E6F0F7CFE5F0F6CFE4F0A2
:100CF000F5CFE3F0F4CFE2F0F3CFE1F072D7E96A99
:100D0000EA6A0C6A086A096A0A6A0B6A04500510E2
:100D10000610071006E1046A056A066A076A30EFE2
:100D200007F0C00E0C1606D0D890043605360636ED
:100D300007360C2A07AEF8D70C2AD89008360936A1
:100D40000A360B360750035C08E10650025C05E1E9
:100D50000550015C02E10450005C09E30880045086
:100D6000005E0550015A0650025A0750035AD890A7
:100D700007320632053204320C060C503F0BDDE11F
:100D80000CBC55EC07F00050046E0150056E02508B
:100D9000066E0350076E0850006E0950016E0A502F
:100DA000026E0B50036E0CAE34EF07F055EC07F0FB
:100DB00034EF07F09E0000EE87F0EE6AEE6A87C01F
:100DC00000F088C001F001509F5D02E100509E5D7F
:100DD000D8A01200F4D7A200A2C0D9FFA3C0DAFFA6
:100DE000A4C0F6FFA5C0F7FF000EF76403D008000B
:100DF000F55005D0F6CFE9FFF7CFEAFFEF50000935
:100E000014E0A4C0F6FFA5C0F7FF000EF76403D0FE
:100E10000800F55005D0F6CFE9FFF7CFEAFFEF5015
:100E2000DF6EDE52A44BA52BDBD7000EDF6A12006B
:100E3000A300A6B2FED7A3C0A9FFA5C0A8FF3F0E7E
:100E4000A616D890F2BED880F29EA684550EA76E44
:100E5000AA0EA76EA682A198A694D8B0F28E120010
:100E6000036A026A016A006AE950EA1008E003C0F6
:100E7000EDFF02C0EDFF01C0EDFF00C0EFFF000C71
:100E8000046E042A0406D8B4000CD890003601364B
:100E900002360336F7D7A300A6B2FED7A3C0A9FF38
:100EA0003F0EA616A680A8501200001E011E021EAC
:0E0EB000031E000E002A01220222032212005D
:020000040030CA
:04000000FF38FCFECB
:02000600FBFFFE
:00000001FF
